:0614000002148B0249E614
:01140B0032AE
:0114130032A6
:01141B00329E
:011423003296
:01142B00328E
:031433000242A2D0
:01143B00327E
:011443003276
:03144B000251113A
:03145300021A95E5
:03145B00021D6F00
:011463003256
:03146B0002432514
:011473003246
:01147B00323E
:03148300024D0A0D
:0314E90002148664
:03148600022E052E
:1014EC00AF83E58290F554F0EFA3F075E10490DF43
:1014FC003BE0FFBF01F890F554E0FEA3E0FF90DF66
:10150C0006EEF075E10290DF3BE0FFBF0DF8227EA6
:10151C00007F0090FC48E0FCA3E0FD8E028F03C32B
:10152C00EA9CEB9D503AEE2400FCEF34F0FD90FC6D
:10153C0046E0F514A3E0F5158A828B83C007C0063C
:10154C00C005C004125646AA82AB83D004D005D085
:10155C0006D0078C828D83EAF00EBE00B60F80B3E6
:10156C0022E58290F556F0E0FFE59CC39FF59CE5E3
:10157C009C24FAF59C439E10D2BA22AF9E74EF5F66
:10158C00F59E22AF83E58290F55AF0EFA3F090FC24
:10159C0041E0601390580812439490FC41E0F582AE
:1015AC001243D67582EF2290FC417406F090DF3B1B
:1015BC00E0FFBF130280F6C29190F557E0FEA3E066
:1015CC00FF90FCA8EEF0EFA3F090FCA274F1F0E415
:1015DC00A3F090FC387472F074F3A3F090FCA0E4C8
:1015EC00F0A3F090FC53F090FC9CF090FC52F09027
:1015FC00FC9E04F0E4A3F090FC9D7402F090F55C6A
:10160C00E4F090000012173490F55AE0FEA3E0FFCE
:10161C0090F559E0FD7B007C008D017A00C3EB99BD
:10162C00EC9A50548B02EA75F0F0A42EF9E43FFAD0
:10163C0090F55C74F0F089828A83C007C006C005FF
:10164C00C004C003121734AA82D003D004D005D032
:10165C0006D007EA601B90585AC002124394D0027D
:10166C0090FC41E4F08A82C0021243D6D0028A82F6
:10167C00220BBB00A40C80A190FCABE0FF30E33349
:10168C0090FCA8E0FEA3E0FFEE540F602690FCA8AF
:10169C00E0FEA3E053060F7F007410C39EFEE49F90
:1016AC00FF90FCA8E0FCA3E0FD90FCA8EE2CF0EF72
:1016BC003DA3F090FCA8E0FEA3E0FFC374FF9EE402
:1016CC009F502390FCA8E0FEA3E090DF02EEF09088
:1016DC00DF04E0FF74FC5FF0E0FF74024FF090FC5D
:1016EC00AA7401F0801290FCA8E0FEA3E0FF90DF4A
:1016FC0002EEF090FCAAE4F075E1037E607FEA90C4
:10170C00DF3BE0FDBD130280091EBEFF011FEE4F43
:10171C0070EDD291EE4F700C90FC667413F09058F3
:10172C007212439475820022AF83E58290F55DF0CE
:10173C00EFA3F090F55CE0FF240F500A9058831251
:10174C0043947582FF22EF703E90FC52E4F090FCC3
:10175C0052E0FE90FC9DE0FDC3EE9D502190FC52AA
:10176C00E075F0F1A42472F58274F335F0F583E49E
:10177C00F090FC52E0FE0E90FC52EEF080D090FC0B
:10178C0052E4F07582002290FC41E0FE601DBE0622
:10179C001E90FC52E0601890DF3BE0FEBE1302800E
:1017AC000E90FC417407F07582ED227582ED22904B
:1017BC00FC52E075F0F1A42472FD74F335F0FE8D4B
:1017CC00828E83E0600A90FC667418F07582FE22AB
:1017DC008D828E8374FFF090FC52E075F0F1A4249E
:1017EC0072FD74F335F0FE0DBD00010E7C0090F51A
:1017FC005DE0FAA3E0FB8A148B158C168F037F0037
:10180C008B178F188D828E838CF0C007C0031255F6
:10181C006DD003D00790FCABE0FE20E3030218DC94
:10182C0090FC52E075F0F1A42472FD74F335F0FED7
:10183C000DBD00010E90FC7DEBF0EFA3F08D828EC0
:10184C008312528BAE8290F55CEEF090FCABE0FF15
:10185C00530704BF043F90FC52E075F0F1A42472CE
:10186C00FD74F335F0FF0DBD00010F8E037C00906D
:10187C00FCABE0FA5302F090FC81EDF0EFA3F0909A
:10188C00FC83EBF0ECA3F090FC85EAF08D828F8367
:10189C001252C5803B90FC52E075F0F1A42472FD0D
:1018AC0074F335F0FF0DBD00010F7C0090FCABE034
:1018BC00FB5303F090FC88EDF0EFA3F090FC8AEE64
:1018CC00F0ECA3F090FC8CEBF08D828F8312530E16
:1018DC0090FC52E075F0F1A42472FE74F335F0FF25
:1018EC0090F55CE0FD8E828F83F090FC52E0FF0F50
:1018FC0090FC52EFF090FC9DE0FEEFB5060590FCDD
:10190C0052E4F075820022AF83E58290F55FF0EF30
:10191C00A3F090FC41E0FF6014BF0102800F9058CF
:10192C009D12439490FC41E0F5821243D612158728
:10193C0090FC4AE4F0A3F090FC4AE0FEA3E0FF8E9A
:10194C00828F83121A1590DF3BE0FFBF0DF890DFFA
:10195C003AE0FF53077FBF6000402790FC4AE0FE4F
:10196C00A3E0FF0EBE00010F90FC4AEEF0EFA3F0D7
:10197C00D29190000A124F91C29190000A124F918D
:10198C0080B590FC417402F090FC67E0FCA3E0FD94
:10199C00A3E0A3E090FC4CECF0EDA3F090F55FE03D
:1019AC00FEA3E0FF90FC50EEF0EFA3F02290FC4180
:1019BC00E4F090FC67E0FCA3E0FDA3E0A3E090FC66
:1019CC004CECF0EDA3F02290FC417404F090FC6719
:1019DC00E0FCA3E0FDA3E0A3E090FC4CECF0EDA355
:1019EC00F02290FC417405F090FC54E4F0A3F090CC
:1019FC00FC67E0FCA3E0FDA3E0A3E090FC4CECF062
:101A0C00EDA3F075820002156DAF83E58290F56150
:101A1C00F0EFA3F090F561E0FEA3E0FFEE2400F5FB
:101A2C0082EF34F0F583E0FF7E008F828E83021408
:101A3C00ECAF83E58290F563F0EFA3F090F563E0F3
:101A4C00FEA3E0FF90F370EEF0EFA3F0222290FCE7
:101A5C004AE0FEA3E0FF0EBE00010F90FC4AEEF040
:101A6C00EFA3F0C3EE9470EF9403400790FC4AE4AC
:101A7C00F0A3F090FC4AE0FEA3E0FFEE2400F58218
:101A8C00EF34F0F583E0F58222C021C0E0C0F0C055
:101A9C0082C083C007C006C005C004C003C002C01A
:101AAC0001C000C0D075D00090FC3DE02401F0A333
:101ABC00E03400F090FC42E0FEA3E0FF90FC3DE03F
:101ACC00FCA3E0FDECB5060BEDB5070790FC3DE47F
:101ADC00F0A3F090FC3DE0FEA3E0FFBE0005BF00CC
:101AEC0002800BBE0105BF00028068021C5790FCEF
:101AFC003DE0FEA3E08E077E00AC9C7D00EC420630
:101B0C00ED420790FC4EEEF0EFA3F090FC4AE0FEA5
:101B1C00A3E0FF0EBE00010F90FC4AEEF0EFA3F025
:101B2C0090FC48E0FCA3E0FDC3EE9CEF9D400790C9
:101B3C00FC4AE4F0A3F090DF3BE0FFBF1303021D6F
:101B4C005290FC4AE0FEA3E0FF8E828F83121A159E
:101B5C00021D5290FC41E0FFBF05028003021D52A2
:101B6C00900019124F9190F567741CF090FC4AE0AC
:101B7C00FEA3E090F568EEF090FC4AE0A3E090F54F
:101B8C0069F090F56A7442F090F56B744CF090F536
:101B9C006C7441F090F56D7448F090F56E7442F0F1
:101BAC0090F56F744CF090F5707441F090F5717481
:101BBC0048F090F5727442F090F573744CF090F517
:101BCC00747441F090F5757448F090F5767442F0A9
:101BDC0090F577744CF090F5787441F090F5797439
:101BEC0048F090F57A7442F090F57B744CF090F5D7
:101BFC007C7441F090F57D7448F090F57E7442F061
:101C0C0090F57F744CF090F5807441F090F58174F0
:101C1C0048F090F5827420F090FC56741CF0E4A30C
:101C2C00F090FC58F0A3F090FC5AF0A3F090F568FB
:101C3C0012465F90FC54E0FEA3E0FF0EBE00010FC5
:101C4C0090FC54EEF0EFA3F0021D5290FC41E0FF2B
:101C5C00BF03028065BF04028008BF050280030237
:101C6C001D5290FC4CE0FEA3E0FF90FC67E0FAA351
:101C7C00E0FBA3E0FCA3E0FD8E008F01E4FEFFEA95
:101C8C00C398FAEB99FBEC9EFCED9FFDC374649A30
:101C9C00E49BE49CE49D50229058CB12439490FC1E
:101CAC00417405F090FC67E0FCA3E0FDA3E0FEA30B
:101CBC00E0FF90FC4CECF0EDA3F090FC53E075F0E1
:101CCC00F1A42472FE74F335F0FF8E828F83E060F2
:101CDC0075900019124F9190FC53E075F0F1A4240B
:101CEC0072FE74F335F0FF90DF04E05401FDB40193
:101CFC0000E4332EFDE43FFC8E828F83E090FC5693
:101D0C00F0E4A3F090FC58F0A3F090FC5AF0A3F090
:101D1C008D828C8312465F90FC53E075F0F1A42405
:101D2C0072F58274F335F0F583E4F090FC53E0FF28
:101D3C000F90FC53EFF0BF0200400590FC53E4F011
:101D4C009058E9124394D0D0D000D001D002D003E7
:101D5C00D004D005D006D007D083D082D0F0D0E00C
:101D6C00D021323290FC41E4F090FC52F090FC53C4
:101D7C00F090FC4AF0A3F090FC467453F0E4A3F00E
:101D8C0090FC487453F0E4A3F090FC4EF0A3F09058
:101D9C00FC4CF0A3F090FC427406F0E4A3F090FC31
:101DAC0044F0A3F090FC50F0A3F090FC54F0A3F09E
:101DBC0012151B90FC41E4F0759DDC859E9E439EA4
:101DCC000443CB1022021D709021F812334D90FC6D
:101DDC0067E4F0A3F0A3F0A3F0121DD190F583E417
:101DEC00F090F5847432F074F8A3F02290FC41E08A
:101DFC00FFBF000302212DBF0103021FFEBF020320
:101E0C00021EFCBF030302212DBF040302212DBFC0
:101E1C00050302210EBF060122BF40028006BF410E
:101E2C000280422275E10490DF3BE0FFBF01F89095
:101E3C00DF0374E5F090DF047404F090DF07741294
:101E4C00F090DF08E4F090DF147410F090DF17E0EE
:101E5C00FF74C04FF090FC417441F090F5847432E3
:101E6C00F074F8A3F090F583E4F090FC54E0FEA33A
:101E7C00E0FF90F583E0FDFB7C00C3EB9EEC9F50F4
:101E8C004590DF06EDF075E10490DF3BE0FFBF010C
:101E9C00F875E10290DF3BE0FFBF0DF890000212F5
:101EAC004F9190F584E0FEA3E0FF90F583E02EFEC9
:101EBC00E43FFF90DF3AE0FD8E828F83F090F58354
:101ECC00E02401F080A475E10490DF3BE0FFBF014A
:101EDC00F890FC54E0FEA3E08E3375340090F5844A
:101EEC00E0F535A3E0F536753201758243022E37E5
:101EFC00E50F7003021FEC90FC65740DF0AF9A7443
:101F0C00FE5FF59AE50F20E403021FEC90FC417490
:101F1C0003F090FC3FE0FEA3E08E8212156D90580A
:101F2C00F712439490FC3FE0FEA3E0FF8E828F8378
:101F3C001243F190F831E025E0FEE42432FFEE3458
:101F4C00F8FE8F828E8312439490F831E0FFB40137
:101F5C0000E433FF90F583F0EF2436FDE434FCFE0F
:101F6C008D828E83E0707290DF04E0FE30E0378F5C
:101F7C0006EE2EFDE42432F582ED34F8F583E0FE16
:101F8C008E337534008F06EE2EFDE42432FEED34D4
:101F9C00F8FD74012EF535E43DF536753201758288
:101FAC0042122E37802290DF02E0FE8E33E4F534AD
:101FBC00EF2FFEE42432FFEE34F8FE8F358E3675AB
:101FCC003201758242122E3790F583E0FF2436F5EC
:101FDC0082E434FCF5837401F0AF0F74EF5FF50FFE
:101FEC00D20010AF02C200750F00A20092AF439A4C
:101FFC000122E50F70030220FC90FC65740DF0AF1C
:10200C009A74FE5FF59AE50F20E4030220FC90F829
:10201C0031E0FF90F583B40100E433F090590C12D9
:10202C00439490F583E025E0FEE42432FFEE34F88F
:10203C00FE8F828E831243F190F583E025E0FEE45F
:10204C002432FFEE34F8FE8F828E8312439490F884
:10205C0031E0FFB40100E433FF90F583F0EF243658
:10206C00FDE434FCFE8D828E83E0707290DF04E020
:10207C00FE30E0378F06EE2EFDE42432F582ED348F
:10208C00F8F583E0FE8E337534008F06EE2EFDE4FA
:10209C002432FEED34F8FD74012EF535E43DF536B1
:1020AC00753201758242122E37802290DF02E0FEDB
:1020BC008E33E4F534EF2FFEE42432FFEE34F8FED9
:1020CC008F358E36753201758242122E3790F5831C
:1020DC00E0FF2436F582E434FCF5837401F0D20081
:1020EC0010AF02C200AF0F74EF5FF50FA20092AFFA
:1020FC00D20010AF02C200750F00A20092AF439A3B
:10210C00012290FC54E0FEA3E0FF90FC48E0FCA30D
:10211C00E0FDC3EE9CEF9D50012290FC417404F055
:10212C0022E50F70012290FC65740DF0E50F543020
:10213C0070012290F831E0FFB40100E433FF90F518
:10214C0083F0EF2436FDE434FCFE8D828E83E06058
:10215C00030221E590DF04E0FE30E0378F06EE2E1F
:10216C00FDE42432F582ED34F8F583E0FE8E337510
:10217C0034008F06EE2EFDE42432FEED34F8FD74AF
:10218C00012EF535E43DF536753201758242122E7D
:10219C0037803590FC97E0E0600A90FC9AE0FDA354
:1021AC00E0FE800890DF02E0FCFD7E00EF2FFCE4F7
:1021BC002432FFEC34F8FC8F358C367532018D33BC
:1021CC008E34758242122E3790F583E0FF2436F55B
:1021DC0082E434FCF5837401F0D20010AF02C2002B
:1021EC00AF0F74CF5FF50FA20092AF2290F7E3E030
:1021FC00FDA3E0FEA3E0FF90F7E8E0FCBC42028008
:10220C0003022B9390F7E9E0FC24BE5003022B85CC
:10221C00EC240A83F582EC244683F583E4738585EC
:10222C00FE4685B16C8A9DD60F3376148585DA59B6
:10223C0080F3182B970B4085858585858585EA73FA
:10224C00BAB0D38585858585858585858585858584
:10225C008585858585858585858585858585AEE896
:10226C002B2B22252B2324242424252525262B2BFC
:10227C00282929292A2A2A28292B2B2B2B2B2B2BB3
:10228C002A2B2A29292B2B2B2B2B2B2B2B2B2B2B98
:10229C002B2B2B2B2B2B2B2B2B2B2B2B2B2B2B2B82
:1022AC002222C007C006C005121587D005D006D063
:1022BC000790FC417440F08D828E838FF01257A5ED
:1022CC00FC7B0090FC54ECF0EBA3F090F809EDF0E3
:1022DC00EEA3F07582011240E6022B9390FC41E4D0
:1022EC00F090F809EDF0EEA3F07582011240E602D1
:1022FC002B9390FC41E06009905926124394022BD9
:10230C00938D828E838FF01257A5FC7B0090F586FF
:10231C00ECF0EBA3F08D828E83A3E0FAE4F92CFCB5
:10232C00EA3BFB90F586ECF0EBA3F08D828E83A359
:10233C00A3A3A3E0FA8A0889098D828E83A3A3A3A1
:10234C00A3A3E0FAE42508F508EA3509F50990FCA1
:10235C003AE4F0A3F074062DF9E43EFA90FC56EC46
:10236C00F0EBA3F090FC58E4F0A3F090FC5AE508D5
:10237C00F0E509A3F089828A83C007C006C0051264
:10238C00465FAC82D005D006D0078D828E838FF04D
:10239C00EC12560E90F809EDF0EEA3F075820112D6
:1023AC0040E6022B938D828E838FF01257A590FC02
:1023BC009AF0E4A3F08D828E83A3E0FB7C0090FC6A
:1023CC009AE0F9A3E0FA90FC9AEC29F0EB3AA3F02E
:1023DC0090FC9AE0A3E090FC9AE0F5F0A3E045F0C5
:1023EC00604B90FC977401F090FC98E0A3E090FC9B
:1023FC0098E0F5F0A3E045F0704712459890FC9AF0
:10240C00E0FBA3E0FC90FC98EBF0ECA3F090FC98C4
:10241C00E0FBA3E090DF02EBF090DF04E0FC74FC47
:10242C005CF0E0FC74024CF012454E801490FC976A
:10243C00E4F090FC98F0A3F090FC9AF0A3F0124515
:10244C009890F7E8E0FC90F7E9E0F53275359A756D
:10245C0036FC7533017534008C82122E37022B93A7
:10246C008D828E838FF01257A590FCABF090F809FB
:10247C00EDF0EEA3F07582011240E6022B9390F87A
:10248C000974ABF074FCA3F07582011240E6022BC8
:10249C009390FCABE0FC5304F090FC797406F09044
:1024AC00FC7AECF08D828E838FF0C007C006C005DD
:1024BC00125233D005D006D00790F809EDF0EEA3F8
:1024CC00F07582101240E6022B9390FCABE0FC53AB
:1024DC0004F090FC797404F090FC7AECF08D828E10
:1024EC00838FF0C007C006C005125233D005D0064A
:1024FC00D00790F809EDF0EEA3F07582101240E6CB
:10250C00022B938D828E838FF01257A590FCACF02A
:10251C00E0FC74015CF090F809EDF0EEA3F075822C
:10252C00011240E6022B9390F80974ACF074FCA3F2
:10253C00F07582011240E6022B938D828E838FF010
:10254C001257A5FC7B008C828B83C007C006C0058C
:10255C00121A3DD005D006D00790F809EDF0EEA385
:10256C00F07582011240E6022B9390FC41E0601C56
:10257C008D828E838FF074EF12560E90F809EDF069
:10258C00EEA3F07582011240E6022B938D828E83AE
:10259C008FF01257A5FC7B0090F586ECF0EBA3F0C6
:1025AC008D828E83A3E0FAE42CFCEA3BFB90F5864B
:1025BC00ECF0EBA3F08D828E83A3A3E0FA90FC3AAF
:1025CC00E4F0A3F074032DF8E43EF990F557ECF029
:1025DC00EBA3F090F559EAF088828983C007C00616
:1025EC00C00512158FAC82D005D006D0078D828E17
:1025FC00838FF0EC12560E90F809EDF0EEA3F07507
:10260C0082011240E6022B938D828E838FF012573B
:10261C00A5FB7C0090F586EBF0ECA3F0EB4C600393
:10262C0002271C90FCA8E0A3E090FCA8E0F5F0A326
:10263C00E045F0601C90DF3BE0FABA1314900028E0
:10264C00C007C006C005124F91D005D006D0078038
:10265C00D290FCA8E0A3E090FCA8E0F5F0A3E04544
:10266C00F0606B90594BC007C006C00512439490A4
:10267C00FCA8E0F9A3E0FA89828A831243F190F373
:10268C0072E0F5821243D690F463E0F5821243D6E1
:10269C00D005D006D00790FC667412F08D828E8324
:1026AC008FF074EC12560EC291C007C006C0051212
:1026BC004529D005D006D00790FC41E4F090F809EC
:1026CC00EDF0EEA3F07582011240E6022B93C2915D
:1026DC0090FC41E4F08D828E838FF012560E90594F
:1026EC005FC007C006C00512439490FC3AE0F9A302
:1026FC00E0FA89828A831243F1D005D006D0079084
:10270C00F809EDF0EEA3F07582011240E6022B936E
:10271C0090FC41E0FABA0602806190596FC007C084
:10272C0006C005124394D005D006D00790FC66E095
:10273C00FABA121B8D828E838FF074EC12560E90A7
:10274C00F809EDF0EEA3F07582011240E6801F90BF
:10275C00FC667417F08D828E838FF074EF12560E18
:10276C0090F809EDF0EEA3F07582011240E6C291EB
:10277C0012452990FC41E4F0022B9374012DF9E4ED
:10278C003EFA90F55CEBF089828A83C007C006C0E4
:10279C0005121734AC82D005D006D0078D828E83FB
:1027AC008FF0EC12560E8D828E838FF01257A5FB94
:1027BC00EC603BBBFE028036905978C007C006C067
:1027CC0005124394D005D006D0078D828E838FF0EE
:1027DC001257A5F582C007C006C0051243D6C29198
:1027EC00124529D005D006D00790FC41E4F090F8B2
:1027FC0009EDF0EEA3F07582011240E6022B938DE9
:10280C00828E838FF01257A5FB7C0090F586EBF03F
:10281C00ECA3F0C374F09BE49C50199058831243C2
:10282C009490F8097486F074F5A3F0758201124047
:10283C00E6022B9390FC52E075F0F1A42472F9742B
:10284C00F335F0FA89828A83E06019905985124336
:10285C009490F8097486F074F5A3F0758201124017
:10286C00E6022B938B0089828A83E8F090FC52E07D
:10287C0075F0F1A42472F974F335F0FA09B900017A
:10288C000A890A8A0B750C0074012DF9E43EFA8949
:10289C00148A157516008B178C18850A82850B8384
:1028AC00850CF012556D90FC52E0FC0C90FC52EC37
:1028BC00F0BC0200400590FC52E4F090F8097486DC
:1028CC00F074F5A3F07582011240E6022B938D8211
:1028DC008E838FF01257A5FC7B0090FC46ECF0EB3E
:1028EC00A3F090FC46E0F9A3E0FAC374709C740367
:1028FC009B402E74022DFBE43EFC8B148C1575163C
:10290C000089178A1890F00075F00012556D90F838
:10291C00097446F074FCA3F07582021240E6022B97
:10292C009390F80974A6F07459A3F07582081240BC
:10293C00E6022B9390FC46E0FBA3E090F8097400B0
:10294C00F074F0A3F08B821240E6022B93121A5A09
:10295C007B008B83121A1590FC4AE0FBA3E0FC90E1
:10296C00F809EB2400F0EC34F0A3F075820112406E
:10297C00E6022B938D828E838FF01257A5FC7B0081
:10298C008C828B83C007C006C0051214ECD005D016
:10299C0006D00790F809EDF0EEA3F0758201124015
:1029AC00E6022B93758200C007C006C00512156D98
:1029BC00D005D006D00790F809EDF0EEA3F07582A3
:1029CC00011240E6022B93C007C006C00512158702
:1029DC00D005D006D00790F809EDF0EEA3F0758283
:1029EC00011240E6022B938D828E838FF01257A535
:1029FC00FC7B0090FC42ECF0EBA3F090F809EDF0BE
:102A0C00EEA3F07582011240E6022B9390F8097444
:102A1C0042F074FCA3F07582041240E6022B938DF5
:102A2C00828E838FF0C007C006C005124353D005B9
:102A3C00D006D0078D828E838FF01257A5F582C0F9
:102A4C0007C006C0051243D6D005D006D0078D822C
:102A5C008E838FF01257A5FC7B008C148B158B1674
:102A6C007517158B1890FC4175F000C007C006C097
:102A7C000512556DD005D006D00790F809EDF0EE93
:102A8C00A3F07582151240E6022B9390FC3DE0FBFF
:102A9C00A3E0FC90FC44EBF0ECA3F090F80974413B
:102AAC00F074FCA3F07582151240E6022B938D8214
:102ABC008E838FF01257A5FC7B008C828B83C00712
:102ACC00C006C005121913D005D006D00790F8091E
:102ADC00EDF0EEA3F07582011240E6022B9390FC10
:102AEC0067E0F9A3E0FAA3E0A3E090FC4CE9F0EA7C
:102AFC00A3F08D828E838FF01257A5FC90FC41F0D1
:102B0C0090FC41E0FBEC24FA404DEB2B2B902B1D61
:102B1C0073022B2F022B2F022B2F022B51022B5126
:102B2C00022B40C007C006C005121587D005D00681
:102B3C00D0078023C007C006C0051219EED005D0FF
:102B4C0006D0078012758200C007C006C00512159A
:102B5C006DD005D006D00790F809EDF0EEA3F07516
:102B6C0082011240E6802090F8097441F074FCA3B5
:102B7C00F07582011240E6800E90F809EDF0EEA39C
:102B8C00F07582011240E6900000222290F7F1E0ED
:102B9C00FFBF013990F7D1E0FEA3E0FF90F7F4E01E
:102BAC00FCA3E0FD90F7D4E0FAA3E0FBEA4B601D38
:102BBC008E828F83E0F9A3AE82AF838C828D83E902
:102BCC00F0A3AC82AD831ABAFF011B80DF90F7DA59
:102BDC00E054FDF090DE11E0FF74084FF022AE825D
:102BEC00AF83E0FD20E703022CE38E828F83A3E00A
:102BFC00FD601DBD0102802ABD0202803BBD0302A7
:102C0C00805ABD04028076BDFE03022CA5022CE383
:102C1C0075370275380090FC6575F0001230E502CE
:102C2C002CE390DE00E0FD7C007539288C3A8D8217
:102C3C008C83123159022CE38E828F83A3A3E0FC88
:102C4C00A3E0FD74062EF582E43FF583E0F539A38D
:102C5C00E0F53A8C828D83123159807B8E048F057E
:102C6C007B0074062EF582E43FF583E0F537A3E094
:102C7C00F5388C828D838BF01230E5805A90F7D129
:102C8C00E0FBA3E0FCA3E0FD753910753A008B82E4
:102C9C008C838DF0123159803E74022EFEE43FFF7E
:102CAC007D00756BAE756C59756D807514048D1542
:102CBC008E828F838DF012505DE5828583F045F016
:102CCC006012D29190012C124F91C29190012C1252
:102CDC004F91800375C9839000002290DF2FE4F0A0
:102CEC0090DF30F090DF31F090DF00740CF090DF6B
:102CFC0001744EF090DF0274FFF090DF037440F02B
:102D0C0090DF04E4F090DF05F090DF06F090DF0731
:102D1C007406F090DF08E4F090DF097424F090DF83
:102D2C000A743AF090DF0B74F1F090DF0C74CAF077
:102D3C0090DF0D74A3F090DF0E7401F090DF0F7430
:102D4C0023F090DF107411F090DF117436F090DFE7
:102D5C00127407F090DF13740FF090DF147418F0F6
:102D6C0090DF1514F090DF16746CF090DF1774037D
:102D7C00F090DF187440F090DF197491F090DF1A26
:102D8C007456F090DF1B7410F090DF1C74E9F09017
:102D9C00DF1D742AF090DF1EE4F090DF1F741FF02B
:102DAC0090DF237488F090DF247431F090DF257469
:102DBC0009F090DF2E74C0F090DF07C4F090DF09AB
:102DCC007425F090DF0A7495F090DF0B7455F09039
:102DDC00DF1A74B6F090DF1B7410F090DF1C74EAED
:102DEC00F090DF1D742AF090DF1EE4F090DF1F746A
:102DFC001FF0221250DF02510B122DFF12443B1216
:102E0C0051381230B01245D1121DD41230DFD2AF6E
:102E1C00122F82D291900002124F91C29190000A0F
:0B2E2C00124F91124117121DF880F8A0
:1058080043616E6E6F742063616C6C207472616E9C
:10581800736D69745F6C6F6E67207768696C65205B
:105828004648535320486F7070696E67206F722026
:10583800616C72656164792070726F6365737369F6
:105848006E67207472616E736D69745F6C6F6E67DA
:1058580021004D41435F7478282920726574757260
:105868006E6564206572726F72006E65766572206F
:10587800656E7465726564205458004648535378C1
:105888006D6974206D65737361676520746F6F202F
:105898006C6F6E67004648535320737461746520BB
:1058A800656E746572696E672053594E4348494E58
:1058B800472066726F6D2077726F6E672073746110
:1058C80074650053594E43485F4D41535445522027
:1058D8002D3E2053594E43494E474D41535445524E
:1058E8000046485353786D697420646F6E65006E86
:1058F8006574776F726B207061636B657428737958
:105908006E6329006E6574776F726B207061636BCC
:10591800657428646973636F7665727929006372A8
:1059280061702C20706C6561736520757365204605
:10593800485353786D6974282920696E73746561BA
:1059480064210064726F706F75742066696E616C93
:1059580020776169742100746F74616C20627974B6
:1059680065732074783A00756E64657272756E009E
:10597800627566666572206572726F72007374690B
:105988006C6C2077616974696E67206F6E2074682B
:1059980065206C617374207061636B6574004E4F91
:0B59A800204445414C005253544E0077
:102E3700AF827E0190DE0E7405F090FC657412F08F
:102E4700E53345347003022F787C107D2790DE111F
:102E5700E0FB30E00D90FC667401F01CBCFF011D27
:102E670080EBEC4D7014D2919003E8124F91C29110
:102E77009003E8124F9190FFFF22BE012C7E009035
:102E8700DE2A7440F0EFF0E532F0AC337D00ECF071
:102E9700E534F0C3743B9533E4953450067C3B7DB1
:102EA70000801AAC33AD348014C374409533E49575
:102EB7003450067C407D008004AC33AD34748025EB
:102EC7002942D6852682852783AA35AB368B01E929
:102ED700F0852682852783A3EAF0852682852783C6
:102EE700A3A374DEF0852682852783A3A3A3742A70
:102EF700F0852682852783A3A3A3A3A3ECFBF085F4
:102F07002682852783A3A3A3A3E054E0F085268226
:102F1700852783A3A3A3A3A3A3A3E0543F4440F01F
:102F2700852682852783A3A3A3A3A3A3A3E054CFC6
:102F3700F0E52942D6E52942D7E52955D160FAE5DA
:102F470029F452D190DE0E7405F090DE11E0FB7487
:102F5700014BF0E533C39CF533E5349DF534EC259F
:102F670035F535ED3536F53690FC657413F0022EE0
:102F77004790FC657414F090000022E5227005125A
:102F8700411780F722AFBE747F5FF5BE43BE8090C6
:102F9700DE0B7407F090DE077411F090DE0914F071
:102FA700438C10AF8C74FE5FF58CD2BD439A0275CB
:102FB7008900C2C5758B00C2E843A90243B90285DF
:102FC7002682852783A3A3A3A3E054E0F085268266
:102FD700852783A3A3A3A3A3A3E0549F4420F0853D
:102FE7002682852783A3A3A3A3A3A3A3E04408F072
:102FF700852682852783A3A3A3A3A3A3A3E054FCC9
:103007004401F090DE01E0FF74FE5FF0E4F525F582
:1030170023F524F52290DE0EF090DE107408F09070
:10302700DE13F090F7DBE4F090F7DAF090F7CFF0EB
:10303700A3F090F7D17488F074F5A3F0E4A3F090AF
:10304700F7D4F0A3F090F7D6F090F7D7F090F7D831
:10305700F0A3F090DE0E7405F090DE107408F09087
:10306700DE13F090DE12E0FF74014FF090DE15E002
:10307700FF74014FF090F7EDE4F090F7ECF090F764
:10308700E1F0A3F090F7E374C8F074F5A3F0E4A3BC
:10309700F090F7E6F0A3F090F7E8F090F7E9F090FA
:1030A700F7EAF0A3F0439A02221244658582288545
:1030B70028F005F07401800225E0D5F0FBF529E53D
:1030C7002875F008A42419F52674F835F0F527902B
:1030D700FC657402F0022F8CD29022C29022AFF0CE
:1030E700AE83E58290F7F6F0EEA3F0EFA3F090F74A
:1030F700DBE06034D2919003E8124F91C2919003C4
:10310700E8124F91D2919003E8124F91C291900328
:10311700E8124F91D2919003E8124F91C291900318
:10312700E8124F9190FFFF2290F7F6E0FDA3E0FE33
:10313700A3E0FF90F7CCEDF0EEA3F0EFA3F090F74C
:10314700CFE537F0E538A3F090F7DB7401F0900096
:103157000022AF83E58290F7F9F0EFA3F090F7DB59
:10316700E06034D2919003E8124F91C2919003E846
:10317700124F91D2919003E8124F91C2919003E8B8
:10318700124F91D2919003E8124F91C2919003E8A8
:10319700124F9190FFFF2290F7F9E0FEA3E0FF7D29
:1031A7000090F7CCEEF0EFA3F0EDA3F090F7CFE5AA
:1031B70039F0E53AA3F090F7DB7401F090000022B4
:1031C7007F0290DE0EE4F090F7CFE0FDA3E0FEC3B0
:1031D70074409DE49E50047C4080048D047F0A8CDB
:1031E700027B00EDC39AFDEE9BFE90F7CFEDF0EE6C
:1031F700A3F08C06EE603690F7CCE0FBA3E0FCA3CF
:10320700E0FD8B828C838DF01257A590DE20F09025
:10321700F7CCE0FBA3E0FCA3E0FD0BBB00010C90A7
:10322700F7CCEBF0ECA3F0EDA3F01E80C790DE1116
:10323700E04FF090F7CFE0FEA3E0FF4E700590F768
:10324700DBE4F02290F7DB7402F07582002290F73E
:10325700D1E0FDA3E0FEA3E0FF90DE11E0FCB401A6
:1032670000E433FC20E0F290DE0EE4F090DE16E09E
:10327700FC7B0090F7D4ECF0EBA3F090F7DAE0FCDE
:1032870030E11390F7DB7403F090DE11E0FC740477
:103297004CF090FFFF2290F7DAE04402F090F7D469
:1032A700E0FBA3E0FCC374409BE49C501CD29190CC
:1032B700012CC007C006C005124F91C29190012C86
:1032C700124F91D005D006D00790F7D4E0FBA3E0CA
:1032D700FC8D07EB4C601690DE20E0FD8F828E831D
:1032E700F0A3AF82AE831BBBFF011C80E6E52C4534
:1032F7002D6009852C82852D8312148990F7D4E0DF
:10330700FEA3E0FFC3EE9440EF9400501DE52A456D
:103317002B6009852A82852B8312148990DE11E0A0
:10332700FF74084FF090F7DBE4F090DE11E0FF74D4
:10333700404FF090F7D4E0FEA3E08E82F58322851C
:10334700822E85832F22858230858331227537012E
:1033570075380090002575F0400230E5AFF0AE8378
:10336700E58290F7FBF0EEA3F0EFA3F090F7FBE018
:10337700FDA3E0FEA3E0FF74022DFDE43EFE8D8277
:103387008E838FF01257A5FDA31257A58D257522A1
:103397000122AF827DEF7E598D828E83A3E090F765
:1033A700FEF0AC1490F7FEE0FBBBFF02803EEBB5EE
:1033B7000723EC700890F7FE74FFF080E71C8D82FE
:1033C7008E83E02DFDE43EFE8D828E83A3E0FB908D
:1033D700F7FEF080CF8D828E83E02DFDE43EFE8DDB
:1033E700828E83A3E0FB90F7FEF080B88D828E83F8
:1033F70022AFF0AE83E58290F7FFF0EEA3F0EFA3E4
:10340700F090F7FFE0F53DA3E0F53EA3E0F53F744C
:1034170002253DFAE4353EFBAC3F8A828B838CF074
:103427001257A5F8A31257A5F9893B753C007402FA
:10343700B53B06E4B53C0280227407B53B06E4B50C
:103447003C028002804274AF58FE7F008A828B83E1
:103457008CF0EE12560EA3EF12560E8A828B838CD7
:10346700F01257A5FAA31257A5F5828A14123399B9
:10347700AE82AF8390F802EEF0EFA3F08E828F83D7
:10348700A3A3E0FE7F00801C89828814123399ACC5
:1034970082AD8390F802ECF0EDA3F08C828D83E08F
:1034A700FCFE7F007406253DFBE4353EFCAD3F8BFB
:1034B700828C838DF01257A5FCA31257A5FDC3EC90
:1034C7009EED9F50048C068D07EE4F700990DE111C
:1034D700E0FD74204DF090F802E0FCA3E0FD8E398A
:1034E7008F3A8C828D8302315990DE0EE4F090DEA4
:1034F70011E0FF30E40E90F7DBE4F090DE11E0FE20
:1035070074804EF0EF30E22490DE11E4F090FC6618
:103517007404F090F7DBE4F0D291900014C0071226
:103527004F91C291900014124F91D00790F7DBE0B2
:10353700FEBE0319D291900032C007124F91C2917B
:10354700900032124F91D00790F7DBE4F090F7DB51
:10355700E06003023830EF20E00302383090DE0EDF
:10356700E4F090DE16E0FFFE7B407C007D40EE60DD
:103577001690DE20E0FA8B828C838DF012560EA314
:10358700AB82AC831E80E7E540FE20E703023703EA
:1035970074605EFD6015BD20030236BDBD400302A9
:1035A70036C9BD60030236EE023818741F5EFF701D
:1035B70041AD41BD0002801CBD06028005BD082645
:1035C700800C90004075F0401233F802381812331F
:1035D700540238187537027538009059CD75F08048
:1035E7001230E502381890004075F040124352023D
:1035F7003818BF0145AD41BD00028005BD0A2680D0
:10360700127537027538009059CD75F0801230E584
:103617000238187537017538009059D075F0801247
:1036270030E502381890DE11E0FD74204DF090006F
:103637004075F040124352023818BF0236AD41BD03
:1036470000028008BD120302381880127537027510
:1036570038009059CD75F0801230E502381890DEA9
:1036670011E0FD74204DF090004075F04012435278
:10367700023818BF032BE4B54112753702753800BD
:103687009059CD75F0801230E502381890DE11E0C0
:10369700FD74204DF090004075F0401243520238FF
:1036A7001890004075F04012435290DE11E0FD740F
:1036B700204DF002381890DE11E0FD74204DF00225
:1036C7003818E52E452F60131236D4800BC02EC054
:1036D7002F90004075F0402202381890004075F096
:1036E7004012384702381890DE11E0FD74204DF083
:1036F70090004075F04012435202381874605EFD26
:103707006015BD20030237CFBD40030237E3BD601C
:1037170003023806023818741F5EFF7048AE41BEB8
:103727000103023818BE0303023818BE0502800BD6
:10373700BE0703023818BE0917800990DE00E5426C
:10374700F002381890004075F040123363023818C1
:1037570090004075F04012435290DE11E0FE742055
:103767004EF0023818BF0129AE41BE0103023818D6
:10377700BE0303023818BE110302381890004075C3
:10378700F04012435290DE11E0FE74204EF00238F2
:1037970018BF0220AF41BF01028076BF03028071CC
:1037A70090004075F04012435290DE11E0FF742004
:1037B7004FF0805D90DE11E0FF74204FF0900040E5
:1037C70075F040124352804990004075F040124313
:1037D7005290DE11E0FF74204FF08035E52E452F23
:1037E70060121237EE800BC02EC02F90004075F08C
:1037F7004022801D90004075F0401238478012909B
:10380700DE11E0FF74204FF090004075F040124346
:103817005290DE11E0FF74404FF0E54645477009CE
:1038270090DE11E0FF74084FF090F7DBE0FFBF0177
:10383700031231C790F7DBE0FFBF020302325522C4
:10384700AFF0AE83E58290F804F0EEA3F0EFA3F0BB
:1038570090F804E0FDA3E0FEA3E0FF8D828E838F46
:10386700F01257A5FC20E7030239A174012DFAE4F1
:103877003EFB8F048A828B838CF01257A5FC601E57
:10388700BC0102802BBC0202803CBC03028073BCDB
:10389700040302393EBCFE0302395B023A0775375F
:1038A7000275380090FC6575F0001230E5023A07A2
:1038B70090DE00E0FC7B007539288B3A8C828B8385
:1038C700123159023A0774022DFAE43EFB8F048A3B
:1038D700828B838CF01257A5FAA31257A5FB7406A7
:1038E7002DF8E43EF98F04888289838CF01257A55E
:1038F700F539A31257A5F53A8A828B8312315902FB
:103907003A078D028E038F048A488B498C4A7406C6
:103917002DF8E43EF98F04888289838CF01257A52D
:10392700F537A31257A5F538854882854983854A17
:10393700F01230E5023A0790F7D1E0FAA3E0FBA3D3
:10394700E0FC753910753A008A828B838CF012314E
:1039570059023A0774022DFAE43EFB8F0490FC6B80
:1039670074D2F07459A3F07480A3F075140475151C
:10397700008A828B838CF012505DE5828583F04547
:10398700F06012D29190012C124F91C29190012CAC
:10399700124F91806B75C983806690F7F1E0FCBC8C
:1039A700015674022DFDE43EFE8D828E838FF01248
:1039B70057A5FDA31257A5FE90DE0EE4F090DE1684
:1039C700E0FF7C007513088F828C83C007C006C098
:1039D70005C004124FDDD004D005D006D007EF4C48
:1039E700601690DE20E0FB8D828E83F0A3AD82AE61
:1039F700831FBFFF011C80E690F7DAE054FDFFF05C
:103A07009000002290F7ECE0FF30E10A90FC66742A
:103A170005F090FFFF2290DE0E7405F090DE16E0B1
:103A2700FF8F4B754C0090DE17E0FCE4254BF54B00
:103A3700EC354CF54C90F7EAE0FCA3E0FD4C7058F0
:103A470090F7E6E4F0A3F090DE2AE090F7E8F09034
:103A5700DE2AE090F7E9F090DE2AE0FD7C0090F79F
:103A6700EAEDF0ECA3F090DE2AE0FAE4FB2DFDEAA4
:103A77003CFC90F7EAEDF0ECA3F0E54B24FCF54BAA
:103A8700E54C34FFF54CC374049D74029C500990B7
:103A9700F7EA7404F003A3F0E52955D16012D29137
:103AA700900014124F91C291900014124F9180E828
:103AB70090F7E3E0FBA3E0FCA3E090F7E6E0FAA3CE
:103AC700E0FFEA2BFBEF3CFC7480252942D68526D4
:103AD7008285278374DEF0852682852783A3742A4F
:103AE700F0852682852783A3A38C07EFF08526829E
:103AF700852783A3A3A3EBF0852682852783A3A32A
:103B0700A3A3A3A3A3E0543FF0852682852783A31D
:103B1700A3A3A3A3A3A3E054CF4410F074052526C1
:103B2700FEE43527FF90DE16E0FD8E828F83EDF0F1
:103B370074042526FEE43527FF90DE17E08E828F7A
:103B470083541FF5F0E054E045F0F090F7E6E0FE0F
:103B5700A3E0FFEE254BFCEF354CFDC374049C74CA
:103B6700029D500B7404C39EF54B74029FF54CC322
:103B77007440954BE4954C502890FC667406F09081
:103B8700DE14E0FD74FE5DF0751304900005124F1E
:103B9700DD751310854B82854C83124FDD90FFFE38
:103BA70022E52942D6E52942D7E54B2EFEE54C3FD3
:103BB700FF90F7E6EEF0EFA3F0E52955D160FAE5BF
:103BC70029F452D190F7E6E0FEA3E0FF90F7EAE090
:103BD700FCA3E0FDC3EE9CEF9D402C90F7ECE04486
:103BE70002F090F7EAE4F0A3F090DE0E7405F0AE71
:103BF7002374BF5524FF8E238F2490DE14E0FF74B7
:103C0700FE5FF09000012290DE0E7405F0AE237483
:103C1700BF5524FF8E238F2490DE14E0FF74FE5FD0
:103C2700F09000002290F7ECE0FF20E1012290F7EE
:103C3700E3E0FDA3E0FEA3E0FF90F807EDF0EEA3BD
:103C4700F090F7E8E0F55474FFB5540280030240A2
:103C5700BE90F7E9E0FBBB800050030240A0EB24D5
:103C67006F50030240A0EB2480FA240A83F582EA0E
:103C7700241583F583E473A035CB08E81F405790DC
:103C870079A0A0A0A0F82B873C3D3E3F3D3F3F3F9A
:103C97003F3F404040403F40408D828E838FF0122F
:103CA70057A5FA74012DF54FE43EF5508A52755326
:103CB7000090F7EAE552F0E553A3F0854F8285506F
:103CC70083E0F5517401254FF554E43550F555A9B6
:103CD700518902E4F92552F552EA3553F55390F725
:103CE700EAE552F0E553A3F0855482855583E0F861
:103CF700854F82855083A3A3884D894EE0FAE4253A
:103D07004DF54DEA354EF54E854D35854E3690F7D6
:103D1700E8E0FA90F7E9E0F5328552338553348AC3
:103D270082122E3790F7EAE4F0A3F00240B68D82B4
:103D37008E838FF01257A5FA8D828E83A38A4D75D5
:103D47004E00E0FA74022DF554E43EF5558A0189D8
:103D570002E4254DF54DEA354EF54EA84DAA4E9095
:103D6700F7EEE8F0EAA3F090F7E6E0F9A3E0FAE966
:103D770024FEF54DEA34FFF54E854D52854E53E549
:103D8700524553603D90F7EEE0F54FA3E0F55074D0
:103D970001254FF9E43550FA90F7EEE9F0EAA3F080
:103DA700855482855583E0FAA3858254858355859A
:103DB7004F82855083EAF0155274FFB552021553AE
:103DC70080BD90F7E8E0FA90F7E9E0F5327535EA5B
:103DD7007536F77533027534008A82122E37024022
:103DE700B690F7ECE0FA20E23C8D828E838FF012DA
:103DF70057A5FA8D828E83A38A4D754E00E0FA90FF
:103E0700F80774022DF0E43EA3F08A018902E4F971
:103E1700254DF54DEA354EF54EA84DAA4E90F7EED5
:103E2700E8F0EAA3F090F7EAE0F9A3E0FA894D8A0F
:103E37004EC37440954DE4954E5006754D40754EF2
:103E470000E9C3954DF9EA954EFA90F7EAE9F0EAE9
:103E5700A3F090F807E0F552A3E0F553854D54859C
:103E67004E55E5544555603D90F7EEE0F54FA3E01C
:103E7700F5507401254FF9E43550FA90F7EEE9F063
:103E8700EAA3F0855282855383E0FAA3858252859F
:103E97008353854F82855083EAF0155474FFB554D8
:103EA70002155580BD90F7E8E0FA90F7E9E0F532A2
:103EB7007535EA7536F77533027534008A82122E26
:103EC700370240B6D291900002C007C006C0051263
:103ED7004F91C291900002124F91D005D006D007A2
:103EE70090F7E8E0FA90F7E9E0F53290F7E6E0F5C9
:103EF70033A3E0F5348D358E368A82122E37024091
:103F0700B67535D77536598B3275330D75340085CF
:103F17005482122E370240B690FC67E0F8A3E0F90E
:103F2700A3E0A3E0883589368B32753304753400F6
:103F3700855482122E370240B67535BC7536598BBB
:103F470032753311753400855482122E370240B60C
:103F570090F7E6E0F533A3E0F5348B328D358E36F6
:103F6700855482122E379000C8124F911244850251
:103F770040B67535B37536598B32753309753400CC
:103F8700855482122E370240B68D828E838FF012AF
:103F970057A5FC74012DF9E43EFABC0202800ABC65
:103FA70003028021BC0429800DC002C00112454EC6
:103FB700D001D002801AC291C002C001124598D028
:103FC70001D002800BC002C00112456FD001D002A0
:103FD70090F7E8E0FC90F7E9E0F53290F7E6E0F5D6
:103FE70033A3E0F53489358A368C82122E370240A6
:103FF700B690F7EA7401F0E4A3F07535367536DF4D
:1040070090F7E8E0FC90F7E9E0F53290F7EAE0F5A1
:1040170033A3E0F5348C82122E3790F7EAE4F0A34D
:10402700F00240B68D028E048C017C0090FC6B740C
:10403700E5F07459A3F07480A3F07514098C158A00
:104047008289838CF0C007C006C00512505DE582E7
:104057008583F0D005D006D00745F0705275C9802A
:1040670090F7E8E0FC90F7E9E0F53290F7E6E0F545
:1040770033A3E0F5348D358E368C82122E37802FA0
:1040870090FC65E4F090FC66F090F809EDF0EEA383
:10409700F07582021240E6801690F7E6E0F533A34A
:1040A700E0F5348B328D358E36855482122E37905B
:1040B700F7ECE054FDF022E5304531601985308298
:1040C700853183121489AE82AF83EE4F701090F75B
:1040D700ECE054FDF02290F7ECE054FDFFF022E510
:1040E7008290F80BF090F7ECE054FDF090F7E8E0E1
:1040F700FF90F7E9E0F53290F80BE0FE8E33753468
:104107000090F809E0F535A3E0F5368F82022E37E7
:10411700E52330E01175220274FE5523FEAF248E8D
:10412700238F2443BE01E5235406602F90FC65745A
:104137000AF075220374FD5523FEAF248E238F24C6
:1041470090DE01E0FF74044FF0900008124F919049
:10415700DE01E0FF74FB5FF075220190DE0EE4F0F4
:1041670090DE11E0FF30E21A90DE11E0FF74DB5FB2
:10417700F090F7CFE4F0A3F090F7D4F0A3F090F726
:10418700DBF090DE0E7405F090DE11E0FF30E520E5
:1041970090DE11E0FF74CF5FF090FC667408F0903A
:1041A700F7E1E4F0A3F090F7E6F0A3F090F7EDF075
:1041B70090DE14E0FF30E62090DE14E0FF749F5F8E
:1041C700F090FC667408F090F7E1E4F0A3F090F744
:1041D700E6F0A3F090F7EDF0E52320E2057404B5CF
:1041E7002214122F8C90FC65740BF074FB5523FE80
:1041F700AF248E238F24E52330E4111234F074E7C3
:104207005523FE740F5524FF8E238F24E52430E6B3
:104217005490FC65740CF0123A0BAE82AF83BEFE6D
:1042270041BFFF3E90F80C7406F0E4A3F090F7E866
:10423700E0FF90F7E9E0F53275350C7536F8753320
:10424700027534008F82122E3790F7E8E0FF75353C
:104257000C7536F87532017533027534008F82128A
:104267002E37123C2CE52354E07006E52454BD603C
:104277002990FC667409F0751308900044124FDD0D
:10428700852382852483751310124FDD741F5523F0
:10429700FE74425524FF8E238F2422C0E0C082C0C3
:1042A70083C007C006C005C004C0D075D000E5BEF6
:1042B70030E6FB90DE06E0FF7E00E5234207E524BB
:1042C70042068F238E2490DE02E0FDE4CDC4CD6D3F
:1042D700CD54F0CD6DFCED4207EC42068F238E24C2
:1042E70090DE04E025E0FCE4FD4207EC42068F2364
:1042F700EEF52430E11290F7ECE054FEF0AE2374B3
:10430700FD5524FF8E238F24758B00C2E8D0D0D0B3
:1043170004D005D006D007D083D082D0E032C0E0E9
:10432700C007C0D075D000E5BE30E6FBC2AFE58957
:1043370030E703752203AFBE74FC5FF5BE758900D5
:0C434700C2C5D2AFD0D0D007D0E03222E7
:1059B300534443437633353000444F4E53444F4EA4
:1059C300474C45207230343530000000000000524F
:1059D30053544E00554E494D504C454D454E54453C
:1059E300440052455345545F4E4F57001201100176
:1059F30000000040501D48600001010203010A0637
:105A03001001000000400100090220000101008094
:105A1300FA090400000200000100070585024000A6
:105A23000107050502400001040309040C035200A9
:105A33006600430061007400180344006F006E00A9
:105A43007300200044006F006E0067006C00650067
:0C5A53000A03300030003900330000FF6F
:10435300AF83E58290F80EF0EFA3F090F80EE0FE45
:10436300A3E0FF7C007D008E028F038A828B83E0B3
:10437300F9A3AA82AB83E960070CBC00EE0D80EBC6
:104383007532F08C338D348E358F367582FE022E66
:1043930037AF83E58290F810F0EFA3F090F810E0C8
:1043A300FEA3E0FF7C007D008E028F038A828B8355
:1043B300E493F9A3AA82AB83E960070CBC00ED0D7B
:1043C30080EA8E358F367532F08C338D347582FEEC
:1043D300022E37E58290F812F07535127536F875AE
:1043E30032F17533017534007582FE022E37AF83C7
:1043F300E58290F813F0EFA3F07535137536F87571
:1044030032F27533027534007582FE022E37AF82A5
:10441300AE83ADF0FC90F815EFF0EEA3F0EDA3F052
:10442300ECA3F07535157536F87532F375330475ED
:0844330034007582FE022E37F1
:0514E400E4F50DF50E1A
:10443B007E197FF88FD57E197FF88ED47E217FF879
:10444B008FD37E217FF87F008ED28F147515188F36
:10445B001690F81975F00002554E7403B50D06E46D
:10446B00B50E02800280047582FF22AE0DAF0E05E1
:10447B000DE4B50D02050E8E822290DF46E0FFBFE4
:10448B00F00E90DF47E0FFBF0D0690DF487469F038
:10449B00C2AF759A0075B80075A8001230E2AFBEB6
:1044AB00747F5FF5BE75D69FC29102000022125534
:1044BB00C2AC82AD83AEF0FFC004C005C006C0071E
:1044CB009037BD75F086743D12544AAC82AD83AE05
:1044DB00F0FFE58124FCF581E4C0E0C0E074C0C0CE
:1044EB00E07441C0E08C828D838EF0EF1256E2AC0B
:1044FB0082AD83AEF0FFE58124FCF5818C828D8348
:10450B008EF0EF1255D5AC82AD83AEF090DF09EE95
:10451B00F08D0390DF0AEBF090DF0BECF02275E1EE
:10452B000490DF3BE0FFBF01F890FC3CE0F5E1902D
:10453B00FC3CE0FFBF04012290DF3BE0FFBF010228
:10454B0080ED2290FC3CE0FFBF02012290DF13E0E4
:10455B00FF74F05FF0E0FF740F4FF090FC3C7402BF
:10456B00F002498D90FC3CE0FFBF03012290DF136A
:10457B00E0FF74F05FF0E0FF740A4FF090FC3C74C6
:10458B0003F0F5E190DF3BE0FFBF13F82290FC3C1A
:10459B00E0FFBF04012290DF13E0FF74F05FF0AF88
:1045AB009174EF5FF59175E10490DF3BE0FFBF0184
:1045BB00F8AF9B74FC5FF59BAFE974EF5FF5E99087
:1045CB00FC3C7404F02290FC3FE4F0A3F090FC322E
:1045DB00F0A3F090FC34F0A3F053C6C7759D008593
:1045EB009E9E439E0485A9A943B90190FC3C74048B
:1045FB00F0751400751500F51690F83275F0001271
:10460B00554E122CE7D2A87591D175E900750F00A4
:10461B00439A0175E10490DF3BE0FFBF01F8227E76
:10462B00007F00C3EE94DCEF9405502490DF3CE058
:10463B00FD5450600490000122900032C007C00668
:10464B00124FBFD006D00774322EFEE43FFF80D34B
:10465B0090000022AF83E58290FC5CF0EFA3F0901A
:10466B00FC5EE4F090DF02E0FF90DF3BE0FEBE1368
:10467B000BB291C007124117D00780EDC29190FC8D
:10468B00AAE4F090FC58E0FDA3E0FE90FCA0EDF056
:10469B00EEA3F090FC5AE0FBA3E0FC90FCA6EBF041
:1046AB00ECA3F090FC56E0F9A3E0FA90FCA2E9F041
:1046BB00EAA3F090FCA4E9C39BF0EA9CA3F090FC66
:1046CB00A4E0FBA3E0FC8D148E158B828C83C007BA
:1046DB00C006C005C002C001125629AB82AC83D004
:1046EB0001D002D005D006D00790FCA8EB29F0EC46
:1046FB003AA3F0E94A705D90FC5CE0FBA3E0FC8B15
:10470B00828C83E0F8881075110090FC56E510F050
:10471B00E511A3F090DF04E0F8530003B80002802A
:10472B0018B8010280030247F190FC567401251062
:10473B00F0E43511A3F00247F190FC5C74012BF00F
:10474B00E43CA3F090FC56E0FBA3E0FC90DF02EB13
:10475B00F00247F190DF04E0FC530403BC0002803D
:10476B0046BC010280030247F190FC5CE0FBA3E036
:10477B00FC90FC5FE9F0EAA3F090FC617401F0E4BB
:10478B00A3F08B828C83C007C002C001124F3CD0B8
:10479B0001D002D00790FC5CE0FBA3E0FC89008B0E
:1047AB00828C83E8F0803FED4E603690FCA8E0FDF4
:1047BB00A3E090DF02EDF090DF04E0FE74FC5EF00E
:1047CB0090FCA8E0FDA3E0FEC374FF9DE49E50099E
:1047DB0090DF04E0FE74024EF090FCAA7401F080AE
:1047EB000590DF02E9F0D2A890FCABE0FE20E303DA
:1047FB0002491F90DF04E0FE530603BE010690FC46
:10480B005E7401F090FC5EE0FE90FC5CE0FCA3E0CB
:10481B00FDEE2CFAE43DFB90FC56E0F8A3E0F9909A
:10482B00FC7DE8F0E9A3F08A828B83C007C006C049
:10483B0005C00412528BAA82AB83D004D005D006DC
:10484B00D00790FCABE0F9530104B90448C007EE64
:10485B002CF8E43DF990FCABE0FF5307F090FC81A2
:10486B00E8F0E9A3F090FC83EAF0EBA3F090FC8571
:10487B00EFF088828983C007C006C005C004C0035F
:10488B00C0021252C5D002D003D004D005D006D03E
:10489B0007D0078046C007EE2CF8E43DF990FCAB3F
:1048AB00E0FF5307F090FC88E8F0E9A3F090FC8A56
:1048BB00EAF0EBA3F090FC8CEFF088828983C007C1
:1048CB00C006C005C004C003C00212530ED002D0F4
:1048DB0003D004D005D006D007D007EE601E90FCA5
:1048EB00ABE0FE5306F0BE50098C828D837410F042
:1048FB0080228A068C828D83EEF0801890FCABE0D0
:10490B00FE5306F0BE500890DF027410F080059045
:10491B00DF02EAF090FC5CE0FDA3E0FE90FC38EDDA
:10492B00F0EEA3F090FC9EE4F0A3F075E1037D6044
:10493B007EEA90DF3BE0FCBC1302801C1DBDFF0137
:10494B001EED4E6013B291C007C006C00512411791
:10495B00D005D006D00780DAD291ED4E700690FCD0
:10496B00667413F090DF3BE0FEBE130BB291C007F1
:10497B00124117D00780EDC29190DF02EFF07582E4
:10498B000122D2A875140075150075160290F83225
:10499B0075F00012554E90FC32E4F0A3F090FC340D
:1049AB00F0A3F090FC36F090FC3704F090F831E473
:1049BB00F0AF9B74FC5FF59BAFE974EF5FF5E975A6
:1049CB00E10290DF3BE0FFBF0DF84391102290FC1A
:1049DB00AD7401F02290FCADE4F022C021C0E0C028
:1049EB00F0C082C083C007C006C005C004C003C0AE
:1049FB0002C001C000C0D075D00090FC657411F0EE
:104A0B00C28990DF3BE0FFBF0D028003024B30D227
:104A1B009190FC97E0E0602A90FC98E0FEA3E0FF09
:104A2B0090FC98E024FFFCA3E034FFFD90FC98EC95
:104A3B00F0EDA3F074FF2F400990DF04E0FF74FC4E
:104A4B005FF090FC3C7402F090F831E025E0FEE45E
:104A5B002432FFEE34F8FEE075F002A42432FC742D
:104A6B00FC35F0FD8C828D83E0FAA3E0FB74012A08
:104A7B00F8E43BF98C828D83E8F0E9A3F0EA2FF59B
:104A8B0082EB3EF583E5D9F090F831E075F002A4A6
:104A9B002432F58274FC35F0F583E0FEA3E0FFC30E
:104AAB009402501A90F831E075F002A42432F5828A
:104ABB0074FC35F0F583E0FEA3E0FF4E701A90F81E
:104ACB0031E0FF75F002A42432F58274FC35F0F569
:104ADB008374FFF07401A3F090FC98E0A3E090FCCA
:104AEB0098E0F5F0A3E045F06003024CED90FC97E5
:104AFB00E0E07003024CED90FC9AE0FEA3E0FF9027
:104B0B00FC98EEF0EFA3F090FC98E0FEA3E090DFB2
:104B1B0002EEF090DF04E0FF74FC5FF0E0FF740244
:104B2B004FF0024CED90DF3BE0FFBF13028003021E
:104B3B004CED90FCAAE0E07003024C7E90FC4EE042
:104B4B00FEA3E0FF0EBE00010F90FC4EEEF0EFA3B4
:104B5B00F090FC9EE0FEA3E0FF90FCA2E0FCA3E043
:104B6B00FDEEB50406EFB505028003024C5190FC37
:104B7B00A0E0A3E090FCA0E0F5F0A3E045F06037E7
:104B8B0090FCA0E0FEA3E0FFBEFF05BF0002801477
:104B9B0090FCA0E024FFFEA3E034FFFF90FCA0EE0E
:104BAB00F0EFA3F090FCA6E0FEA3E0FF90FC9EEEDE
:104BBB00F0EFA3F0024C5190FCA2E0F514A3E0F54A
:104BCB001590FC9CE0FF7E008F828E83125629AEDF
:104BDB0082AF8390FC38E0FCA3E0FDEE2CF582EF76
:104BEB003DF583E4F090FC9CE02401F0E0FF90FCA9
:104BFB009DE0FEEFB5060590FC9CE4F090FCA2E076
:104C0B00F514A3E0F51590FC9CE0FF7E008F828EDF
:104C1B0083125629AE82AF8390FC38E0FCA3E0FDF3
:104C2B00EE2CFEEF3DFF8E828F83E0701090FC41E7
:104C3B00E4F090FC667412F0124529C29190FC9E30
:104C4B007401F0E4A3F090FCA8E0FEA3E0FF90FC5D
:104C5B00A8E024FFFCA3E034FFFD90FCA8ECF0EDF2
:104C6B00A3F0BEFF22BF001F90DF04E0FF74FC5FC8
:104C7B00F0801490FCA8E024FFFEA3E034FFFF902B
:104C8B00FCA8EEF0EFA3F090FC3C7403F090FCA2B8
:104C9B00E0F514A3E0F51590FC9CE0FF7E008F82FD
:104CAB008E83125629AE82AF8390FC9EE0FCA3E06C
:104CBB00FD90FC9EE02401F0A3E03400F0EC2EFE0E
:104CCB00ED3FFF90FC38E0FCA3E0FDEE2CF582EF0E
:104CDB003DF583E0F5D990FC3AE02401F0A3E034F4
:104CEB0000F0D0D0D000D001D002D003D004D0053A
:104CFB00D006D007D083D082D0F0D0E0D02132C004
:104D0B0021C0E0C0F0C082C083C007C006C005C090
:104D1B0004C003C002C001C000C0D075D000751222
:104D2B000090FC657410F0AE9B74FC5EF59BE5E99E
:104D3B00420FE5E930E02090FC3DE0FDA3E08D065D
:104D4B007D00AB9C7C0090FC3FED4BF0EE4CA3F058
:104D5B00AEE974FE5EF5E9E5E954707003024EEDC1
:104D6B0090FC3CE0FEBE030AAE0F748F5EF50F02A3
:104D7B004EE690F831E0FEB40100E4332436F582C0
:104D8B00E434FCF583E0FEBE01028003024EC390C7
:104D9B00FCABE0FE20E103024E9C90DF04E0FE53EF
:104DAB000603BE010375120190FCABE0FE53060136
:104DBB00BE017090F831E025E0FDE42432FEED34C5
:104DCB00F8FDAB127C00EB2EFEEC3DFDE0F929FA71
:104DDB00E42432F9EA34F8FAEB29FBEC3AFCE075FF
:104DEB00F002A42432F58274FC35F0F583E0F9A3CC
:104DFB00E0FAA8127F00E9C398F9EA9FFA90FCAB9E
:104E0B00E0FF5307F090FC81EBF0ECA3F090FC83F8
:104E1B00E9F0EAA3F090FC85EFF08E828D831252BD
:104E2B00C5806E90F831E025E0FEE42432FFEE34CD
:104E3B00F8FEAC127D00EC2FFFED3EFEE025E0FA14
:104E4B00E42432FBEA34F8FAEC2BFCED3AFDE07586
:104E5B00F002A42432F58274FC35F0F583E0FAA35A
:104E6B00E0FBA8127900EAC398FAEB99FB90FCAB34
:104E7B00E0F95301F090FC88ECF0EDA3F090FC8A84
:104E8B00EAF0EBA3F090FC8CE9F08F828E83125347
:104E9B000E90F831E0FF74016FF0E0FF75F002A4A3
:104EAB002432F58274FC35F0F583E4F0A3F090FC2A
:104EBB0036F090FC37F0802190FC667412F0B291C2
:104ECB0090F831E0FF75F002A42432F58274FC35C2
:104EDB00F0F583E4F0A3F0B291C291AFE974CF5F28
:104EEB00F5E9E5E930E61490FC667410F0B2911226
:104EFB004529B291AFE974BF5FF5E9E5E930E714F5
:104F0B0090FC667411F0B291124529B291AFE9741D
:104F1B007F5FF5E9D0D0D000D001D002D003D00410
:104F2B00D005D006D007D083D082D0F0D0E0D021EE
:104F3B0032AF83E58290FC63F0EFA3F090FC61E06D
:104F4B00FEA3E0FF90FC63E0FCA3E0FD90FC5FE0C0
:104F5B00FAA3E0FB8A008B011ABAFF011BE8496038
:104F6B0024EE2AF8EF3BF9E82CF8E93DF9EA2CF5A9
:104F7B0082EB3DF583C006C007E088828983F0D0C1
:064F8B0007D00680CF22D2
:105A5F000000000000000100000000000000000036
:075A6F000000000000000030
:104F9100AE82AF831EBEFF011FC3E49E74808FF0FB
:104FA10063F08095F050167C4C7D04EC24FFFAED03
:104FB10034FFFB8A048B05EA4B70F080D722AE8266
:104FC100E583CE25E0CE33FF1EBEFF011FC3E49E65
:104FD10074808FF063F08095F040ED22AE82AF8354
:104FE100D2919003E8C007C006124F91C29190017F
:104FF100F4124F91D006D0071513AD13ED20E754ED
:10500100EE30E024900019C007C006C005124F9190
:10501100D291900226124F91C291900019124F9194
:10502100D005D006D0078022900113C007C006C06A
:1050310005124F91D291900032124F91C29190017D
:1050410013124F91D005D006D007EFC313CE13CE64
:10505100FF1D80A8C2919003E8024F91AFF0AE838B
:10506100E58290FC6EF0EEA3F0EFA3F090FC6EE011
:10507100FDA3E0FEA3E0FF90FC6BE0FAA3E0FBA33D
:10508100E0FCA814A915E8496050C000C0018D8258
:105091008E838FF01257A5F98A828B838CF0125779
:1050A100A5F8E9C398F98916D001D0006010E5167A
:1050B100F5173395E0F518851782851883220DBD04
:1050C10000010E90FC6EEDF0EEA3F0EFA3F00ABA32
:1050D10000010B18B8FF011980AC90000022AFBE8F
:1050E10074FB5FF5BEE5BE30E6FBAFC674B85FF595
:1050F100C6E5C620E6FB43BE04E5BE30E6FB53C66B
:10510100C743E40C43E401D2B92243FE03C2912216
:10511100C0E0C082C083C0D090FC67E02401F0A34E
:10512100E03400F0A3E03400F0A3E03400F0D0D08C
:10513100D083D082D0E032124465AF8290FC75EF0B
:10514100F08FF005F07401800225E0D5F0FB90FCB2
:1051510076F0EF75F008A42419FE74F835F0FF908D
:10516100FC71EEF0EFA3F08E828F83A3A374DFF0C6
:105171008E828F83A3A3A374B1F08E828F83A3A3A6
:10518100A3A3A37410F074062EF582E43FF583E027
:1051910054E0441DF074072EF582E43FF583E0549A
:1051A1003F4440F074072EF582E43FF583E054FC60
:1051B1004401F0124465AF8290FC77EFF08FF00567
:1051C100F07401800225E0D5F0FB90FC78F0EF75DA
:1051D100F008A42419FE74F835F0FF90FC73EEF08A
:1051E100EFA3F08E828F8374DFF08E828F83A3749E
:1051F100B2F08E828F83A3A3A3A3A37410F07406CD
:105201002EF582E43FF583E054E0441EF074072E4E
:10521100F582E43FF583E054CF4410F074072EF596
:1052210082E43FF583E054FC4401F043A91043B903
:105231001022AF83E58290FC7BF0EFA3F0E5B33061
:10524100E3FB90FC71E0FEA3E0FF90FC7BE0FCA39C
:10525100E0FD8C028D038B028E828F83EAF090FC3D
:1052610071E0FEA3E0FF8E828F83A37D00ECF090BE
:10527100FC76E042D690FC79E0FF90FC7AE0FE4FAC
:105281004401F5B3E5B330E3FB22AF83E58290FC43
:105291007FF0EFA3F090FC7FE0FEA3E0FF90FC7DA8
:1052A100E0FCA3E0FDEC540F60158C028D030CBCF7
:1052B10000010DEA2EF582EB3FF583E4F080E68CE8
:1052C100828D8322AF83E58290FC86F0EFA3F0907C
:1052D100FC86E0FEA3E0FF90FC81E0FCA3E0FD90F2
:1052E100FC83E0FAA3E0FB90FC85E0F990FC8FECF5
:1052F100F0EDA3F090FC91EAF0EBA3F090FC93E4C5
:10530100F090FC94E9F08E828F83025358AF83E5CD
:105311008290FC8DF0EFA3F090FC8DE0FEA3E0FF06
:1053210090FC88E0FCA3E0FD90FC8AE0FAA3E0FB9E
:1053310090FC8CE0F990FC8FECF0EDA3F090FC91E7
:10534100EAF0EBA3F090FC937402F090FC94E9F086
:105351008E828F83025358AF83E58290FC95F0EFE4
:10536100A3F0E5B330E3FB90FC95E0FEA3E0FF90F2
:10537100FC8FE0F51AA3E0F51B90FC94E0FB745060
:105381005BF51990FC93E0F94B4401FB740149F57D
:105391001890FC91E0F514A3E0F515E4F516F51766
:1053A100C3E5169514E5179515400122C00390FC3D
:1053B10071E0F8A3E0FBE5162EF9E5173FFA890441
:1053C1008A058D0488828B83ECF090FC71E0FCA34C
:1053D100E0FD8C828D83A3E9F090FC73E0FCA3E0F7
:1053E100FD8C828D83A3A3E516251AFCE517351BD9
:1053F100FD8C028D038B02EAF090FC73E0FAA3E0CE
:10540100FB8A828B83A3A3A3ECF090FC78E0FD9050
:10541100FC76E0FC4D42D6D003E5196017E5142473
:10542100F0FCE51534FFFDECB51609EDB517058562
:1054310018B380028BB3E5B330E3FB74102516F586
:1054410016E43517F5170253A11254EDBC000302FF
:1054510056B4EF60FA30D502B2D1E583B4FF03024E
:1054610056CAE582B4FF030256CA25834007248247
:10547100400B0256B424831450030256CAF582EA43
:105481008DF0A4A8F0EA8EF0A428F8E435F0F9EB49
:105491008DF0A428E935F0F9E433CA8FF0A429F995
:1054A100EA35F0FAEBF88EF0A429F9EA35F0FAE4DE
:1054B10033FBEC8DF0A429F9EA35F0FAE43BFBE883
:1054C1008FF0A42AFAEB35F0FBE433CCFD8EF0A487
:1054D1002AFAEB35F0FBE43CFCED8FF0A42BFBEC5E
:1054E10035F0FC20E70312551B025693AA82AB83C9
:1054F100A2F73392D1F5826002D2F7ACF0E58124B4
:10550100F9F8E6FD08E6FE0886F008E6A2F7339210
:0A551100D5F5836002D2F7AFF02257
:0614BA00E478FFF6D8FD06
:10551B007804EC7011E58224F8500AF582E4C9CACC
:10552B00CBFCD8EF22EC7820058220E713D5820143
:10553B0022C3E933F9EA33FAEB33FBEC33FCD8EA59
:10554B00158222AC82AD83AE15AF16BE0004EF60A0
:10555B000C1F0FE51412560EA3DEFADFF88C828DAA
:10556B008322AD82AE83AFF08D198E1A8F1B8514FB
:10557B001C85151D85161EA817A9188803890418E4
:10558B00B8FF0119EB4C6025851C82851D83851E98
:10559B00F01257A5FCA385821C85831D8D828E83FB
:1055AB008FF0EC12560EA3AD82AE8380CE8519829E
:0755BB00851A83851BF02215
:101498007917E94400601B7A01905A5F7897759331
:1014A800FCE493F2A308B800020593D9F4DAF275C4
:0214B80093FFA0
:1055C200FCABF0AA83A982749EC2D1F58212551B4C
:1055D2000256937F9E1255FC30D1030256B4C3EF9C
:1055E2009582500974FFF5F0F583F5822279001255
:1055F20057C189828A838BF0EC22AA82AB83A2F7FD
:105602003392D1F5826002D2F7ACF02220F711304A
:10561200F6138883A88220F509F6A88375830022F1
:1056220080FEF280F5F022E5828514F0A4C582C0E6
:10563200F08515F0A4D0F025F0C5838514F0A425DB
:1056420083F58322E514451560467A01E51425E0C9
:10565200F514E515334012F515E5829514E58395A9
:105662001540030A80E6C3E51513F515E51413F595
:1056720014C3E5829514F5F0E58395154005F5838D
:1056820085F082C3E51513F515E51413F514DAE177
:0156920022F5
:1014C0007800E84400600A79007593F0E4F309D8E5
:1014D000FC7897E8440C600C790D90F000E4F0A3E0
:0414E000D8FCD9FA61
:02148900E4730A
:10569300B98003EA13B34010EA2401FAE43BFBE4C4
:1056A3003CFC50047C800582BC000EBB000BBA009E
:1056B30008E4F5F0F583F58222A2D1E582138CF09C
:1056C30092F78B838A8222E4F583F58275F080F466
:1056D300A2D11322E4F583F58275F0C0747F221200
:1056E30054ED30D502B2D1BF0009BC00030256D736
:1056F3000256CABC00030256B4E583B4FF0BE5822D
:10570300B4FF030256D70256B4E582B4FF03025630
:10571300CAC395835007247F400B0256B4248014D8
:1057230050030256CAF582C3ED9AEE9BEF9C4011DB
:105733001582C3EA33F9EB33FAEC33FBE433FC8031
:1057430005E4CCCBCAF9C08275F019C3E99DEA9E82
:10575300EB9FEC9400D5F002802D400EE99DF9EA11
:105763009EFAEB9FFBEC9400FCC3B3E833F8E582AD
:1057730033F582E58333F583C3E933F9EA33FAEB8F
:1057830033FBEC33FC80C4B3E4F938FAE43582FB31
:10579300E43583FCD082500405827C8012551B02C1
:0257A30056AB03
:0D148B00758155125804E582600302148635
:1057A50020F71430F6148883A88220F507E6A8832D
:1057B50075830022E280F7E49322E0226040F82519
:1057C50082500274FFF582E824F8501ECCCBCAF94A
:1057D500E4CC24F85014CBCAF9E4CB24F8500BCA16
:1057E500F9E4CA24F8500379002224086010F8C3AC
:1057F500EC13FCEB13FBEA13FAE913F9D8F1227564
:03580500820022FC
:00000001FF
